:100000000C94D31B0C94FB1B0C94FB1B0C94FB1B40
:100010000C94FB1B0C94FB1B0C94FB1B0C94FB1B08
:100020000C94FB1B0C94FB1B0C94FB1B0C94C13419
:100030000C94FB1B0C94FB1B0C94FB1B0C94FB1BE8
:100040000C9434350C94FB1B0C94FB1B0C94FB1B85
:100050000C94FB1B0C94FB1B0C94FB1B0C94FB1BC8
:100060000C94FB1B0C94FB1B7622972272227622A7
:100070007A22972287222F244B24B124442435242A
:100080004E2462248024204C3A0020033A002F00A2
:10009000043A0044494747455200444947474552BE
:1000A00000CF00D800E400DF00C600BB00AF005462
:1000B0006F67676C65204D6F6465004C6576656C95
:1000C00020646F776E004C6576656C207570004E0D
:1000D00065772047616D6500526573756D650053E6
:1000E000617665004C6F6164000008430C46733014
:1000F0000008623398EA2B442088313D0F68ACF445
:100100007A8B61AAF47D1FE7FC7B4B93A85CABF173
:10011000603FDE8F61FF7A3E5953E87F168E1F2BBA
:100120005B9EE908CE660008430C46733000086207
:100130003398EA1B2A418A329D0352A1B43B2E4BCD
:10014000F13B6F8F43C9F9AD8ED88A572AE87FA655
:1001500049DD7AD72D4FD368FA3DC9B9755F0CA137
:10016000154AE14B08430C467330C6318C5192E37B
:10017000A1042210A908A63C184242108019083197
:10018000C3134341507D0DA805515D350887A04F2D
:100190003AC084417C553D43A17C5E068F9837E18F
:1001A000054BA0885F16C7B803E02470320000F842
:1001B00076868425296188CE63084D8865119CC2A6
:1001C000608430C46733000708430C467330C6218F
:1001D0008A219147508E188CE63A9C63294AD000B8
:1001E00000F8239984318765508C1100C20922AA36
:1001F000F81234C414C8AABD142668C4210DB53839
:100200003DA5E8FA97D5ED7C3180C44210206E60A0
:100210000D62A3B24252946368EA1BE1B7803E804C
:100220000F430C3119CCC01F084D0C4673285A00DF
:100230000218048A0684C018C70C4673080C100FF5
:1002400047E64600D421D7E7AF80011108422E28A7
:10025000177260B76825554C127AF81A19C69A2495
:10026000F5F1507B4FC7500C6108C719E3364801C0
:100270000C01B21F71F0633154A7F05F99EF0010C9
:1002800084D0C46732801B08430C467330C4230CEF
:100290006318D7190C24A8AC018AC08C268A9EA0AA
:1002A000AE2A5CA0210C93F3C8341000A0001F0EEE
:1002B000021D409A668FC8E8FC4D97D07602F6651D
:1002C000B094A52946305D2210842FE01F06F1511D
:1002D0006045A8BA01C521B82F8D09A06EC0408421
:1002E00030C46733002808430C4673308421082348
:1002F00010C431086000815355753E818C68FA3016
:10030000E181FC9F486A65FD15004610814A0000A6
:100310000DCF14F9AA7D4021284B3794A50800166B
:10032000C404210840CE00861A00D601208821543A
:10033000CD09EB0168FB0F13A090C1086188CE6660
:100340001408430C467330C6386022108420827033
:100350005D40218AA798834C8B479874407C40F875
:100360006A18E7E1FE0295000008411CF001144103
:10037000ECE8DB9F49538B20887A1084A5297B8287
:1003800086309202100010C024154B81254F7CD876
:10039000150557A1E12608430C4673302108430C8C
:1003A000467330C6386233988D5001421084010084
:1003B0001108003D0123210841906314403A88133D
:1003C000C8EA0A6B18A8C42A829BD1BD88A2C8F9C2
:1003D000FE4AAEA7A86ABF944216D5FCFCA427A18A
:1003E000A97CC218A20F0251F856007F11001B2AE7
:1003F0000421862339981408430C467330C63862AA
:100400003398EA010C510C8A3104221D763294A5EE
:1004100000230A808410C1FFFC2421083055D780B6
:100420004329D4FA0800A00010C461840066D003F8
:100430002C27E20903F18650DA29A21029A88802A4
:1004400004BA3E82412C44FE3EA8CC2211218FC02A
:1004500010C462AF83F88CE6601C08430C4673300E
:100460008422086118C70C46419B02700010C00628
:100470000004206CE2121090C465A20820D3741C02
:100480003F47188628846004A810D3B6E887A00CDC
:1004900070C467318420ABEA638C8B00010C46602A
:1004A00006824A7EA430BEFF9430C467330002083F
:1004B000430C467330C4318E1834773C5413248A6D
:1004C0003A9EDFD1F7FF9DAD437E7FAD84233E7D15
:1004D0001084D1FE66FCFF2789F3D8FF3ECFF3FFDF
:1004E0002BF9C218623399802908430C46733000F7
:1004F000086003908810185505A7C10C63086A228C
:1005000012F88C853406B88E6A29E6A1F23E1A8F5D
:10051000B8A919EC102BF848305A1A26A3BC0E596A
:1005200007C2318E682000050340A8A6800E610234
:100530002492F922D288308822883E1208934D9066
:10054000521485FA33820C84B249C08E68F83F8811
:10055000CE662208430C46733106210000080031A4
:100560000E48962A01CB21A7F4100348088399E886
:100570003C0EA0126A18C043F0780AAC0150000487
:1005800025B1695F5510C55100401441510AA418A6
:10059000C43F634039043F01B508CA518FE1A23C12
:1005A0009084800000025446A96A92547A35511012
:1005B000057C0862AB82219168202208430C4673B7
:1005C000300001000D8CA609E2A008C24B87260866
:1005D0004F390C8009824212A2E8E6008442168656
:1005E0000DC0001848118C631847F0701A12FB04F4
:1005F000791F086B8D0C822089F112AA8C7E33D46E
:100600008120C2008F48902A5F400327F1F3EB2935
:10061000910A3F800057000002188CB2CD939C2DA8
:1006200008430C4673308001108486231000198221
:10063000C40188628864408401008631C3119147F7
:100640005152C2F4000D084426944192A6208432EF
:100650001084E62A7FB2A32687560521EE2E0F804E
:100660007A4104417C06A809F0B74CF8341A87286F
:1006700008008003980034301072C471FC1070C6FA
:10068000E1C44673300E08430C467330C8320C8404
:1006900021C00043000661108E43049351E241CE15
:1006A0005720E857C9382D0B8A0520324604190710
:1006B000F1F0F392B42B0AD8B8F49F428CE4076DA2
:1006C00004031DE388FE1B1E87DC2BF3A8541D03C7
:1006D000D3F2B4118C70C0C9E8AAD937D1B046732F
:1006E000301508430C4673311A408C76E808130421
:1006F0002D2342000171000010571A010928E677E6
:10070000854F9BE8FA8FA3A3F12DA8F51F9F47F90A
:100710003D8CD7E018C798E91F0B6A6CEB520E109E
:100720001B4334917E310C5144673477D275200FCE
:1007300008430C46733340063231000018C5A10946
:1007400026B18863A8C15055402124CA843758C7B0
:10075000A052ADBD32CF8803EE060318C696072C13
:10076000543DD5472D681F3FF6D086B4193B0C0683
:1007700096000421139CF8063182328E75368D7CEA
:100780004774DEA9BF8C4322D0400B08430C46734C
:10079000301A008842108918840069A2800679A660
:1007A0002B09EAA2CAC84112A7F03D2D149A17C31B
:1007B000A00A7A08C638623398EA7B9F4300010C8E
:1007C000463A22EA7A9430C68F4237D0886456E49B
:1007D000357DD7F1F273300708430C467333400080
:1007E000004C10851C4C200841388EB88E8425D4CE
:1007F000231CB0030846D02686681F0E80C8EFE28F
:100800000C30114793E14A529471947810F40C0023
:10081000A328F0210000000E328F2A415471DE8F90
:10082000BFE8FBFE8FBF8421862339982D08430C37
:100830004673300000362900063208841540318E98
:10084000188C2A121084A872B902A1D22A2CD3E0E3
:10085000F62A5E63D06FC42A94C4A434310AA7F880
:10086000A90F9EA5FA3E418C7A2D4AD00000F8854A
:1008700054842BCCB596FCF956A7F108210C3119FC
:10088000CCC01808430C4673318631C31198C53863
:100890006735480006801548AA00547650C1A1AEBD
:1008A000A7B2BE107F048CB9800000A2229A8002F9
:1008B000001A125482A8B432553F3B5B516A175D4F
:1008C0004F54D4FD45464F8E3397271C2400632494
:1008D000B6B5B6AE2BD5001008430C46733084284D
:1008E000606390E71A980018C70C461A3D3D53D52F
:1008F000FA062FF514A5A9FF70840000003192427A
:100900009AAA7ABF47ABC2118C210C73209638A0EB
:100910001AD6C3118719521A9EA800BF0BEA95C2B6
:100920004208430C46733088224311410530884108
:100930000D3B445C36C68320CD559E8342DD7F86C9
:1009400089E05536568010847194AE100010C02492
:100950005000D53D4C0D1EA7F987A3FCE010042FD5
:10096000916221082206389401380421862339989F
:100970001108430C4673300006846310C6419A7315
:10098000A84150888318E7309348A6B50D82A2FE8F
:100990000211933120E7CF81BF0631C84E7508039D
:1009A000F07A239CC378006310E31FE2A2FE03F0F9
:1009B000DA021CFC41D423D0BE06E304A93D90FB1F
:1009C0001F04FBFC7C151AFA00804319249268412D
:1009D000862339980608430C467330C6386233982C
:1009E000EA7B9F42001B1434031B41145493C455EB
:1009F000297C44BC62A94BE2FE23398EA7B9FE20B4
:100A00007C3154A5F136A26D94DF909A0C552803E1
:100A1000E3FE23398C2132EB7A9430C4673300082B
:100A200008430C4673301A0002188F270A80631897
:100A3000C6210A1896AA5A6EABD104221221D4AA52
:100A40007A9F46FBC6D085BF055D30FC9F818C63D5
:100A5000535F2017F853153E85F94A753EA1267C51
:100A600020680008623C6FC01862339980190843FF
:100A70000C46733182418C241104210C8100881AA8
:100A800044600C50410470C79248C2B88A58CC02E6
:100A90005BC67D8207B00800BD47801DB5BCF34032
:100AA000054008C021DC7A8F9420D2221B87C80819
:100AB000C84F8C3208B43A287CC5C410804000036B
:100AC000CD4813C7904D82C008884DD2A09C45D612
:100AD0007A24E67B9916821708430C467330000689
:100AE000C411E4E3506A23DFE890044414303E402C
:100AF00080022A236823A839BF25A122C641C31139
:100B000050BE3D080318E18212A300022A8016009D
:100B1000AA70134106602105B520C6AF245A3B5B7D
:100B200088532427CA10C31190E61D01BEC7E11ED9
:100B30004E397EFE100108430C4673308612046362
:100B4000180678C24810678D62A204B41A0042CC1D
:100B50004798542A00320D03A2D0FF9F845D46B50A
:100B60001E685D4086288790154A5094310943E4F9
:100B70007C0209040002188C7C1F848411041684F2
:100B800044036A3DE3908CFD8FE7BD57FE132E6E44
:100B9000022A4F7FFE3908430C467330180000616B
:100BA00068C63088421049504D1500062A9041C24F
:100BB0000D519061294A5D1EA3003430000068C2C7
:100BC0001092E8C007A04E140109D0CC610884211E
:100BD0000EA4B4042D044418331E83C0A8AC85832E
:100BE00091A9F43EC482D1EA418884B43461545D51
:100BF000C1063D83E888645A081808430C467332DE
:100C0000C00000228C40118C84206381C304AAA6FA
:100C100021548210B53AE340FE22A08267C206301A
:100C2000E46111082D009F493D21869020BE52139A
:100C300041BE7A80C764AA6A6EA1A0DE62AF0F7B54
:100C4000F43E808803113409006307C24FA6A12037
:100C5000EA009A3810BACFE62A95C21708430C4624
:100C60007330C638623318000110218E0153D3024D
:100C700008484A8A39CC0841541FC0471DC9D811B9
:100C80003DDDA42117C0420C4315802A8C84153108
:100C9000A1D524D03F808E3B93B905832C17C9DFA3
:100CA0007C64A8C82159C4AA021079560DA2410C2F
:100CB000C1086188CE661708430C467338426680C7
:100CC0000C001A18C420CE8842430408014CD454A6
:100CD000FD35A0E6E000F5AE2B0CF459ECD381080D
:100CE000FA0F603A2DBDF8FC77D771E054BBC5858B
:100CF000E493ABFE06D88253F8B70CB3A1D0BE86FE
:100D0000F97FD0C0BA82B88CE6601F08430C4673E6
:100D100032C2A00010C4647210810806420E400C5A
:100D2000804103C28C47487F221E2350902408C76D
:100D3000645B138FC55828000431D80B421DC3F0E3
:100D4000E85519350D13502683F0450318F618C3DE
:100D500088D0337D6F19B62FAC6642066FA3242668
:100D6000D04842106209081273FF78400E08430C05
:100D7000467330C8320C8421C00043000661108ED7
:100D800043049351AAF2CE5720E857C9382D0B8A55
:100D900005203246041907F1F0F392742B0AD8B8F3
:100DA000F49F428CE4076D04031DE388FE1B1E873D
:100DB000DC2BF3A8521D03D3F2B4118C70C0C9E828
:100DC000A6D937D1B04673301B08430C467331089F
:100DD00048608200C0338000003381EB600802026B
:100DE0001062A800220C6425F158E31926E7F804E4
:100DF00064F04641CD000431F872150FF1AACBA47E
:100E0000BE04020C879478847C1CC441B88C631F98
:100E1000E1A18F4018079D347A024690924805B2AE
:100E20004203A10F01EC1341FC2A15AB91BC3E0615
:100E3000FD26D0761916822608430C467338C60262
:100E40000C23084841908421299202783DF5915E57
:100E50001A04516084000000808452C54633E85F64
:100E6000090299001E4035826F1545E14058412026
:100E7000B59500000009F0806411067AC7408ABA6F
:100E8000116E59C23F12006318F08A83409AB00B6A
:100E9000E008D126426181098242136148C2AD4017
:100EA0006BF86F9916821E08430C467330842860D5
:100EB0004218000860016042320C9108F9300C01C0
:100EC000094A6294B700484B2001A839DD0AA026E0
:100ED00080AAA8631C303D1098010811673AC7C565
:100EE000598C6002F9206823188411847A58C72429
:100EF0004C12067184080027B20008049A241A8B49
:100F0000E0C27299C44CA9081200426825027A1AFC
:100F10000FF1154AE12608430C46733340000001E7
:100F200058442143118042008E29204842431185B4
:100F30004263597740E21D0748D000004311823ECA
:100F400009A5BA16B119CC23184838A02210842854
:100F5000EA80FC2D0B02DA06124A865820C83204B9
:100F600025F62A0A6360294A5A2000003B9A8A69BA
:100F7000E43E2112A7A80842102320E304CD44E454
:100F80003A88CE662D08430C46733088018C632066
:100F9000641108421042418361204200D318068246
:100FA00090909A05405294A4BC03A20000380041DE
:100FB0008B904CD0007C40EE03F08FF01683508075
:100FC000841590420E401907C8041A1EF1C8DF03A9
:100FD000D6BE11085E40C442461A0109890E61E47A
:100FE00000007156013B12742190341A848909174C
:100FF000580CE6A8BB28F2741808430C46733188D5
:10100000118C03004812340000179C4E208C87D5A9
:1010100003D8A433018E4120C551687E85C16C027E
:10102000A3D07830907FD7A2927C1F9545655D3222
:101030002D43F10D310483385434A56A9A8A76E041
:10104000FE0EDB65F802409221914210C3119CCE46
:101050001108430C4673300000849182E509A49581
:1010600001AB01D8180E31516C2406A1CCE89C5676
:1010700025A4FC5D166DA35F378C9411C984B080E4
:10108000160403D07531EE3B17152DD6170DB5E0BC
:10109000691FA8389D13ABD23F26E758501A10900D
:1010A00084CB364E702208430C467330C638A0926B
:1010B000404710925820C000022A9241700491C803
:1010C0001A0E4760AC421B43D0088420F834054315
:1010D0003C52150621A47C231908422C84F43E8B33
:1010E0002826294B0C0423C0341DA40004303A8860
:1010F0006DF807536502BE2A32108411044127B1EE
:10110000F8071E07E0087A8AA42DF8E33A4ABA9550
:10111000FD801E08430C467330C6318042143119DD
:101120008AA4B22EA8C82121081A9C6B192A0C6027
:1011300001860219A728D0D20002188C2A3FA037B6
:1011400080425294BC8CD51C0C61D683A461249E31
:101150000714D4F90541C6689C9049ED0077854293
:101160006A846127F230704DD012127363492E0BDE
:101170000A3399802808430C4673388421042421BB
:1011800002000218184231D443A86780809510ED00
:10119000A1D40320F439E289001A20887A1F223C66
:1011A00003900E89A9840419218902A10002CF208D
:1011B0006210BA8D0CA50F100A9F43006B827C1A37
:1011C000007E3180440700518C2327C364009500C2
:1011D00001780482F817508426A882426819CC67E7
:1011E00033002A08430C46733106718C848608420A
:1011F0002C751D0129084294482964151DC350927D
:10120000A40001680C4188345A9823F87181085071
:10121000C4635004351761E4467F153F6DFC2528F3
:101220006762530427C21084230E103A9C10C590A5
:10123000421B92C62A6DE63399EB706008430C4658
:101240007332C631C3119CC410921824532149959E
:101250000D83FC4555FE2FD1F6F97D35B5E8F53FF8
:10126000CFF2E8FB97CF46FF3F3E5FF384631C312C
:1012700019CC61086188CE6430401708430C46736E
:10128000300006C411E4E3506A23DFE89004441000
:10129000C621F204001151E8350F37E4B4C458C830
:1012A00038622A168E300C6386084F8C0008AA001C
:1012B0005802A9C04D0419808416D4831ABC9168C1
:1012C000ED6E214C909F28430C4643987406FB1FFB
:1012D000847938E5FBF8401A08430C467333400024
:1012E00000018C2500908400430C04944475D8D4EC
:1012F000399479D1F519800984806318C72CF021BD
:101300009C05408C84BE2E2ACEC015B1F0A80017D3
:10131000F10C00951F0032040308368EE2315D3077
:101320003F42A046E771611281AC81C3138B6F010C
:1013300090840B651000988D614C1251A42E8FB6CD
:101340004EF6000908430C467330863108411908EF
:10135000208000036A318C2118AA12108404D15015
:101360008D63228C19E03148C8305B059EBE9B27F7
:10137000C8BC783EC42155B78D8008C4ADBA2FE4EF
:10138000D12FA8F33AD20E3FE74AC380308F008AAC
:101390006681085B0545E584222089C8814009AE45
:1013A0008D83EE95C21808430C467330C6386042F0
:1013B000BB65100000B2C0A00311A8231DAECCD0A5
:1013C0005B187ABA1F521213D81909886860D06A5C
:1013D0001DF81B893480451F2688119E321AB78C50
:1013E000E01A09347D183B9ABE2B440A00F61D18FA
:1013F0006BF8B6AF80DD97B52B840208430C4673BB
:1014000030C6010C638E06000001862A018EAA9860
:101410000006D73A0671A8E33A8E80218AABEE49DE
:10142000518C9F8FF070F5238C3E098680F9EE90E9
:101430000E21F83218CA70A46A2036D338CE388705
:10144000E0180DC0E8FA10343F13E2EE3E15EC63ED
:10145000CCDBA8DB519CCC0208430C4673318600E0
:1014600080110C863304231D2154466000C7EC0113
:10147000B55363CE63C1D3F9AA986318E9DA9884A7
:10148000A92AFD1FE7DF2A56FF4D8F3DFDDFE1183A
:10149000FF7FE463085750EE3C8F60337D10C467D4
:1014A00033000A08430C4673300008600054AAACAD
:1014B000E16118C618A832079FFE549940C6216CF6
:1014C0005C8801D0D0318926AA6038C0860B2421DF
:1014D0000443FDCD3B5643A08008000000E71900FF
:1014E0001BA2FC1BDCB1DD663A82B603D49A114B19
:1014F000A3108109B4BF94350ECB2B841108430C83
:10150000467330C635C411C4B33812A010850C54CC
:10151000F50E57A11064189B53D46318B46F07E3FA
:10152000A8430C6E7D04F029C4428606529793B8F6
:1015300045C0886000072D705217C001104418C9BB
:1015400051585505E820840108618B0A5C080008A1
:1015500060C12000844D56AE2BD5001608430C46C2
:101560007330C62308631C31300C842540210AA047
:1015700008882A9F20AA2A5DE741268F5267174FC5
:10158000C2296398D02A7A685F01341C8347F846E1
:101590003F07419ABE2AA6A7D03A0DC242D1F41104
:1015A00078BF28844F808427C6BEC7D19168201495
:1015B00008430C467330C431884286231980750075
:1015C000C70C46731E860000085463A2FD1B7FE013
:1015D00010DB54FF51516AFCCD467FF452C689FEA0
:1015E000F9353FF5E568E3184A50D4FA1FC3A3263E
:1015F000A459AA448421862339981208430C4673BF
:101600003000D03400088631C31185414CD51538DF
:10161000424212182686002AA7A93E40C3118FCE47
:1016200010DFA200010C02A310842E2EB9F478D989
:10163000F0213042BFB0199681A817B2D03330D410
:101640002217A3F1211A98692AC3D3FE1BC6F9BF3A
:10165000D01708430C467330000001118108408800
:101660004210B3F08F98A9342DA81530C7C40C7D53
:10167000D54E386072104A5294B53DC97C854A00F7
:10168000000054F5006188CFA09F1AD6C30DF9322F
:101690003F4800E6FE418EB2D097610426A933EEA2
:1016A0002A7A93B5800E08430C46733000086232E4
:1016B00008C4310C5505BE1A687509084204042691
:1016C0008FC80C630806394E60A9BE18A6380B34C3
:1016D000410AA008425284260AB1AF8753B203F4EC
:1016E000FCD586D02AC6D19132AE07A190908479DC
:1016F000779C79EC66FC22F1FDBC200A08430C467D
:101700007332C6318C6168000046610D34308064EC
:10171000180364D40A90C04212A1368FA00C601E38
:1017200089BD23B26D44DD1B58086188C86210A1D1
:101730008B6654D1773E92A7A9C23D5F33A8821829
:1017400060252C99F0B400043119CC196EC9CE0073
:101750000608430C467330C00001B1480631C3038C
:10176000A865C926E2A8895AE055093F2CE1A0E8FE
:10177000175178B48E899154DCCE83CC7719A77138
:10178000F0501CC92A52681DD4E7EC8FE1EE669236
:101790007A55174199C79A10CD9D376AFC4210C3FC
:1017A000119CCC0F08430C467330C6300010C01497
:1017B000001AA410EDCE69B53D440004201AF4507F
:1017C0006855087B8EAEA118EA79CB4307F1DC9708
:1017D000D8EC639093C8B8557454B906838D763E9F
:1017E00007004D080318EE9DA6A3E3C2D084E121B3
:1017F00003106723982721D43AACAE100E08430C8F
:10180000467332C6318C5150850C08610D3351CA74
:1018100058854A0056E10F06211360EAFE024E3455
:101820008F621863E2A0B2CD0FD900002C9B440652
:10183000D1A3D49B007A8084A5D8884D06A08ABE07
:1018400041FC1908BC1DE400001BA0182126177CD0
:10185000E3322D040D08430C4673318000430054DD
:1018600082318C63CF48424304A9FFFD13DC8EAA6A
:10187000520C4317060C29B536F03A83E8054EB9E9
:101880008350DC74668024D1FE2CA2A068000E0474
:10189000611C401210840E703C02D1B8E719E6A515
:1018A000E8552E7C1FC46733000908430C4673308B
:1018B0000008623398426A8357C6A89D11B8854CC8
:1018C000121090C461A3FBFC9FCF3DFE9AFEAFA314
:1018D000F778BF59580002D1F43F9387080752693F
:1018E000FA8800BCBF7F080B08430C467330000821
:1018F0006233988C108F57D1DBAAC9BF068FC9B746
:1019000040C3B47CFF8B1F8042109B4E1221886223
:10191000154BC080631C31A44653D02DBF82A3D089
:1019200082A00000E838AF86682F6615FC2DD0AF86
:10193000AA87B18CE6600A08430C4673310800346C
:101940000004311990210041B3E5551E7FC4E824FD
:10195000D5788F22493670101229FE17766E5C47B3
:10196000CF19802DEEB2DDEF35F3393B97E026E855
:101970004CD344DCB35F335803739F4097E657332F
:10198000001008430C467332C00000028CA3910380
:101990003F084631C303A83381882210BF92FF1A43
:1019A000010000882421218C267809AA2D035CD00F
:1019B0006C9D148318863F8398104639863A907838
:1019C000816E3C0535A061220884216E753E8FA191
:1019D0008002EB3D22FC43A93DB0042186233998C7
:1019E0000C08430C467330C421431180C638602470
:1019F000A825B8F2A7B1F435E9FF18FE110C431081
:101A000038FF9AA1AF2A6A26A7E83F1D04A52C310A
:101A1000A3F520002180C80802A6CA9463BC6B2DE0
:101A200018C32009FD13E60C3119CCC06008430C23
:101A30004673300008623398CD53DDC10908420275
:101A40002A8C249A9EA5B4340FA75AD0EA2F8EBFB1
:101A5000A9F5FF9E21F9FE4A9300F9F4520021F600
:101A60007F9914153817538430C467330005084331
:101A70000C467330C000B1810302C0066010EA1A40
:101A800022B8A2AA59DB40E234158C638623398B35
:101A9000E78C24AF8A8CF8EA496340D62BBD04302A
:101AA000C467327C00002188CE62A875FEACB50800
:101AB000B5FEABE11FF46A9FD7FFC00108430C4697
:101AC00073300E0002188CE61A9ED7D001ABD4FFFB
:101AD000BE8FABFCABA9FFB2689AB8006A9EA7D1D3
:101AE000B55E02A7A9F47D4B62F9FF81807518618C
:101AF00088CE662408430C467332C00043119CC252
:101B000060841A88E2AE98012102024511C302C026
:101B100065151511510218A8863C622AE459A146A0
:101B20001A2543F1F21F27200033E7F8680D13BA96
:101B300066D3E054F3D54FF10E2A947E3DC2219135
:101B40007E10C3119CCC1A08430C467330842104C8
:101B50000000A208EEA71D471C6824D04C63431167
:101B60008D4CC31084860843302108461D1F430056
:101B7000160002188CE60084C62640221B99EE7DD2
:101B800081088230EA0FDAA509064210DFC92A7AF5
:101B900080C0AA6A216886212A9A9C83A62AAF80DF
:101BA00030C46733002D08430C467332C000006315
:101BB0001C3119108108AA7A6C410E73A3909A0DFA
:101BC0004F4E0F47A7AA7A7F4017CD4E0BE7CD7E29
:101BD0007A7EA7CDFE117045F44B529BEA07B329DC
:101BE00098210C3119CCC027318D0C467332C0219D
:101BF00000008CE623180218EA88CE6231863294FF
:101C0000621467315405000B6446730E800055164C
:101C10004467845426357319CC0CF829031AC18CF7
:101C2000E61F8BD1917C0A9EA718084D6633987EDB
:101C30000212A98CE62A92C19148631A188CE660B8
:101C40002C08430C467332C00000E100411085802F
:101C50000042486036056B50D011052F3D54FB956E
:101C6000478BFC4DEEBE8B8A3908E6B004842430E5
:101C7000426F586548CA93C80059A3D45F3E807329
:101C80009CFA3E8FF27B9F01BE10C3119CCC5A0878
:101C9000430C467333000043000864C6CAD53DEACE
:101CA0002030216CA7C80D6318E1819A441842CBFB
:101CB00065989C75C806ED14B94C108486084A8254
:101CC00055A9EA7D1F47F998267CFF3FCFF3FCC159
:101CD000862339982D08430C467332C000430064B4
:101CE0008800042000842862D81005105445A94CAF
:101CF0006318D53E8262108409B47A9024A859F002
:101D0000FF1A210CCF88A5862A6F881FC4626F42F4
:101D1000A7A9299D1F42018C63181F2ED52AD4EC38
:101D2000A9C218623399801308430C467332C0006D
:101D30000042143023088220821A640318E18A6C5E
:101D400095132C20539A2D3FA2E6FA3FE39B0F40B8
:101D5000180210C3119F803F805987F7CD0B2018C0
:101D6000C70C46731842220A2191680A9EE7D1F8EF
:101D7000708430C467330041304218623398CC130A
:101D8000300158C638623103730698000D40218A2D
:101D900099019A10C6154FF54CE212202188C7A868
:101DA000BE097518C68629A25415510848629AA81A
:101DB0007E8A9EA3A6BE7F8A9AF6C84AAAA1A7EAEF
:101DC000BD0337D50211E6FFD8C2608430C4673145
:101DD0009804318D0C46733340C03221914063002A
:101DE000210C3119CC2DD0020002188CC000E85A09
:101DF000BF300D06A1D45B99B341F8350204910FB1
:101E000053A18B000057C48BB8D0778F9F450843F0
:101E10000C467A2615996A5A167FA9FC0D03621999
:101E2000141F01A188CE663C08430C4673308428F9
:101E3000623398EA7B9C21369FA3FDFF30C212C318
:101E4000011C65248420035A0002188C25ACA4814F
:101E5000862339843A08E188CE62D03C693AA7B932
:101E6000F47E1C215FDFF306188CE6603B08430C10
:101E7000467330000030842430424E2CA8C1BB325F
:101E80006A600831D95C88C5859094F004209290EE
:101E9000A82AE154FAAD31A3FF74CFCFFC2E9BF9F1
:101EA000FF9A6FE2184631D5C3184C10800C00021F
:101EB00010C31184C134545A5EE14C330ED5B9803D
:101EC0000708430C4673300008623398EA026BFD42
:101ED000492A1D5F33A8F57CC743D5E6AA9354CCA5
:101EE000B450B5AD6B733A989F3E8DF1FF1F3E69BC
:101EF000AA7C26CFC2137C0BCDF55C7F6F630843B1
:101F00000C4673300008600610850C4621099800C5
:101F100008557D424300031EAF51553ABD49A82FD5
:101F200057A9357D1FFAD5EA4D5F47D5FF8A9B57E4
:101F3000D1F5661747D4FF018421862339981A0802
:101F4000430C46733080001091408231B268054FD7
:101F500051500188748D04431D4240B2B917C3E843
:101F6000D47F00001F869AA9FE3A9EA2143155FC28
:101F7000C2D80355FCB4CD5BF2537A90C6CF8CB473
:101F8000D8005D0BC80849E82FF127C3D032C0083C
:101F90004D194B54100908430C4673300842430254
:101FA000104000430C2540318E188C2A32543FA833
:101FB000FFFBF180D100CD1F47D119B47172868F1C
:101FC000A3E8598E872968FA3F3199E832A68FA392
:101FD000FC19DAC23E10D73E6E102B08430C467334
:101FE00030022080F141E512108BA92CAA8C43A964
:101FF000EA410D9A3ED621F41F3FC54C544301C01F
:102000000C00F14D446094210C5529CE1695F52A0B
:10201000D4F678424001BB0C5529541547C0425EA6
:1020200031449114FC12CCF15206188CE6602A0857
:10203000430C467330842860225822898EA3284698
:10204000318C25A9C451840038023AABE228C15032
:1020500000E10555F0D3150E800AABE0A67403D954
:102060005A88434D0034C545FC0434D68FFC042106
:102070008623007D13732EBF60FCDB308098C1A8DF
:102080004F644C5D4DC23F6003E8FFA8AA57085D4E
:1020900008430C4673310848608218852E54C510D9
:1020A000CB53E8A3D1F451E8FA3E8E10C31188C790
:1020B000338C631922992A51A8A52B92F8E849A1DB
:1020C00000F5EFCE004AB53D45C4FC0BD10FA01082
:1020D0008420CC1086188CE6603008430C4673329E
:1020E000D8318E188CC63030210006210A188CC6D3
:1020F000005444212188CEA5D1F47D1F4728CB1060
:10210000C85F2800086233F946386233D142DD3DAA
:10211000B40D43F19FFAA9F4FD17E337CE186233EB
:1021200099800F08430C467332C20000206C412096
:10213000B2680D00488645A92C1917B0A9EA7D1F81
:1021400047F809F844322FC410C3119CC23F8000E5
:102150008623398F41104510C8BE0000300E2191F2
:102160007402D816C46730FC20043119CC66CDF84F
:10217000704608430C467332C631C3119CC4108CA0
:102180008420C70C5C049AAA1996A2BE343987230E
:102190009A7E0C13C00EC3A0E75A2ED23D0F619158
:1021A0004753F65D1E8731D75A3CC5A4FCF4EEC7F1
:1021B000F3F711C906608430C46733001508430C77
:1021C000467332C0200010C46734042000EAF008CF
:1021D000751D5F4D547AB535527F228629AA9865C0
:1021E0008629BD17DB972A620C64A9E9B0B401AB5C
:1021F0003E426F5567C74C9AAEF8B306772CFEC2C5
:1022000010C3119CCC0A08430C467332C631C30379
:102210001842210C6210821A7472B5407100408815
:1022200003A804151802708020E423BB42A0ACEA86
:1022300046DE390EC3A202A21822118C77DB3FA81A
:10224000AA50187F0A448302B5800C5A96F1515166
:102250001105484A9F48D04B511B434803557C41C8
:10226000862339980608430C46733300CB1E7C0046
:10227000016046110B27AA8A38FEE58A9F52CC34AA
:102280007D406330E4AF88802440358C72E7C17DA7
:102290008C750715F333A0033E6A8821863A8A9F1E
:1022A00032D5345CF751F9335DD31FDBC22F0843BD
:1022B0000C467330C621046100010C46552B4008C2
:1022C00062A718D6321090C467FCEE039066190D11
:1022D0009B88FD1FB732087E7F899517CFFCEE43A0
:1022E000F4BECA97E7F8751F9FFB3781F0FDE10840
:1022F000EA2F9FE3F1FFC01108430C46733000083A
:102300006002910006541A98C77AD100D54206653A
:102310001526D1B05CDF17E6CF9FE70FB6CA9EF94E
:10232000E0BA900A6B188FF4ED1F00C24212180F2A
:10233000A2001FE158CD52501A8FC01D17B8F434B7
:10234000208430C461E9591475AD8C004208430CF7
:10235000467330180002188F278A82E5CBB4020C2E
:1023600084212E08E668D0A62A96E9A9EA7FE430FF
:10237000C48B452800043005C880568FC7FC242133
:10238000218936A224CD6D1347D1FE018C70C4671C
:102390003118210C3119CCC00C08430C467330C6DF
:1023A00031AE2992642084020001149E55D0F613A8
:1023B000834719084860603CABA3AB4708000001A5
:1023C000A0698D144D41086188C4C6EA27CF9407DF
:1023D000F9C7F5006704AB518AA0D024AA8BECD0D2
:1023E0003E6F6FF83CA9F006188CE6600508430CB8
:1023F000467330000862330306318EA1D7FA818C10
:102400005A3F07501327DC7A017C7ABE804A8F67D7
:10241000EC063168FC132A0264FB8FC02F8F57A88B
:102420000951ECFD80C62D1F4418C9648E188CD646
:10243000309BE1F5E6601308430C467332C63088E2
:1024400042108D190678882AC2539526A550E27548
:102450001FF3A0619527F04A73E1EE3FA1F9334ED7
:102460008C30839EA9860BDAA7A9C20034006000D5
:1024700008C9B285414C582100592D5404212182AC
:1024800010671CB81086188CE6601608430C46735B
:1024900032C0000040147449A421884410443565BA
:1024A00042408F601D43A96864D0220FEC9A197EC8
:1024B0000882AB1687895498C6842F8220A6F441DF
:1024C000F703F8C82F08812681105375104210B603
:1024D00028A7342F20409A69BA94661DB751FA3163
:1024E0009CCC1A08430C467332C63188628864005B
:1024F0008C600C5153D4E31974718744ADEA408762
:102500006AD8F4510AB7F819F25D7B07C7ED040CDD
:10251000ACFE32109748000D86A7A85954FC8310D2
:10252000BE008618D18631C3119CC21361BA6F14E4
:102530000F08430C467332C631C3119CC59FF17519
:1025400018CC20883108823A9696A9EA7D0C5A1751
:102550002119FC22F886018221903A0F8EA7C62904
:102560008D1F72EC7D8F9EA10300007C01284B1013
:10257000C818C4421B22E08CC7355BD936D0370857
:10258000430C4673301A000218647734541A8AEEEA
:102590009E607DC36A121090C4C121E823A8C7764B
:1025A000481A3DD9A0FF011C41D0C84CF80006C410
:1025B00011C4AB7D69724C880090848607261B414C
:1025C0001D4616497E4B3DCF864500010C462C8C9E
:1025D000FE0C663399801E08430C4673308631C367
:1025E0000B8EE6810433355D53DCFA3F0FF3FFFFBA
:1025F0000114320C90C4664254241D6098606464D7
:1026000091526803DA374A9BFBD007F14955F544EC
:1026100031C3119CC7531AE708430C46733029088D
:10262000430C467331084088429023C2544318E15A
:1026300088CEA2FA580000638C7FBCB021160798A0
:10264000AF20CE3480F81EC7C1A3789F2D93504988
:1026500077C8BC1A90E09E383EEBE1A10842770DA6
:10266000DA000D8279A92D093B433EE06A9FF98A81
:10267000A570801408430C467332C631C303184654
:1026800001822060434C82A210040886A3D0CA02B3
:1026900080AC2D44C0000CD1F42F47F0D0730D0C4A
:1026A000033545A3E8F99E86C0000CD1FE2CE22933
:1026B0000E67A1D4BA3E820D1F47FEC174440108C3
:1026C0006188CE661A08430C46733084212E280890
:1026D00000086230084631C30318401188629442F2
:1026E0005294A38A2A1BD02DE56A2068518FCB31E2
:1026F000842210A181545F2E7953D4FF0B000FC4A4
:10270000212E8E10F704204368D4B40545F188418A
:10271000002A7F907501806F8830C46733001C08E1
:10272000430C4673300008623398EA7B9F40FDFEFD
:102730007A844221090C465F20C7FFFC03D97FDA67
:1027400020631EC14BCF151340C0442D0546BCA0CD
:1027500007002A80019CC74042102CD02B0A067922
:10276000A8BCCFA2A718C70C46213682186233999D
:10277000801408430C4673310216921818E58190B4
:10278000841D42300C30C54F53E82218F80D1E79D5
:10279000A9FE31713A3FC0127E3EC7517DD420CC94
:1027A000FE11AEF9A89A1034000042508430C4677C
:1027B0003203E0632F8C4328EA2A3B222190EA115E
:1027C000D4F5298210C3119CC61208430C467330FD
:1027D00084286042580008623008657BD42128CAEA
:1027E00052C317BE8FCBFCFC87143E5DBF38421826
:1027F00062336FCC318E188C2FFA87E22049A4DD2A
:1028000055202A0F86A7654062473A3E8FF1061889
:102810008CE6601408430C467332C4000811502241
:10282000A1042300C03146528CE010CDE488718DA4
:10283000189B10B91D0701D1F47FF252D0737BAF02
:1028400042CD774D1731D4F4104BBB1809A014209A
:10285000002188CC00A2291ADC06AC421862339908
:10286000801808430C467331C00200008E23098093
:102870002708690886CAB8288A80328CD1651F0863
:10288000D031FB2AA4D47E7FE731EE2CD1D75AAFCA
:10289000F751747B91F9008EA3F73920AF4127B728
:1028A000A97F3F08799D46E925437CFB7F21821063
:1028B000C3119CCC1E08430C467330000080438635
:1028C0002319E831D0C50C46384E80BD6346D2741A
:1028D0007D18C1FA3F0D1B3AA6B47F9F47EA747D6D
:1028E0001FEC296188C69C0819D0F71C037E4003A1
:1028F000A0ACE4A0848426E3A97713DD2119CCC021
:102900001208430C467332C0310850C466300021AF
:10291000000631C31198EA40430024793C6821083D
:102920006188CE83CBF6DF8B4FD28216E4FBA7C340
:102930009FE623D641FCE5C4A90A52C31198747DD1
:10294000782317C4618C70C46750FF1154AE101700
:1029500008430C4673300006C411E4E3506A23DFD9
:10296000E890044410C621F2040011511B41A879DB
:10297000BF25A122C641C31150BE3D080318E18204
:1029800012A300022A801600AA70134106602105D6
:10299000B520C6AF245A3B5B88532427CA10C31105
:1029A00090E61D01BEC7E11E4E397EFE101A084397
:1029B0000C467333400000018C2500908400430CCA
:1029C00004944475D8D4399479D1F5198009848058
:1029D0006318C72CF0219C05408C84BE2E2ACEC0E3
:1029E00015B1F0A80017F10C0368A8780190201821
:1029F00041B477118AE981FA1502373B8B08940DAF
:102A0000640E189C5B780C84205B288004C46B0ADD
:102A100060928D21747DB277B00A08430C46733101
:102A2000822108421C30318C8D0B42100661A0249B
:102A3000221023A870AA90633D45F554C0A200BFA0
:102A4000B2A7D07E7A9800001A306C41CAAA021050
:102A500080A809B010952723A01E88D619F0B7E9E1
:102A60001B46323746086188CE61F87318AA55CBE9
:102A7000F7F0800108430C46733086120463180691
:102A800078C24810678D62A204B41A0042CC4798FD
:102A9000542A00320D03A2D0FF9F845D46B51E6804
:102AA0005D4086288708154A5094310943E47C022A
:102AB00009040002188C7C1F8484110416844402CB
:102AC000AA3DE3908CFD8FE7BD57FE132E6E022AC0
:102AD0004F7FFE0708430C467330C6210800048070
:102AE00039800010422A86791CB21B82A121084A33
:102AF000E43A8049607C01086180D41F07F01080AF
:102B0000000003A1E4388802088318CC3C0C26A0FE
:102B10006D43FC6B039A342D846125323D03E2D171
:102B2000AA1CE7E007C24184440B400012A6D0442F
:102B3000100C60E6160203E018C44207386E81FCF0
:102B4000454697C00B08430C467330000880920C32
:102B5000B118D4521DF0102AA33D93A31F98F85525
:102B6000BC06F23FB582E79EC68398721A9F17A3F0
:102B7000F1212687899FF85681AD68FC81EE0D050D
:102B80005AB607A3CE5D1680626A1782F91CC09FF1
:102B900007951E4E801408430C467330842860420B
:102BA00008E5318C2118C70C4A15385A00006321FA
:102BB0002EEA8644A9E609E03A1CA5F0DCE30B5BAB
:102BC00014548010484EA2A206D40A8893C02A50FA
:102BD000543F3E834C7C0AB4368F8E99F8C953819A
:102BE0007529A18185A1086188CE66110842688295
:102BF000388CE621086318844210220B48D23738FB
:102C000050AC0A80231869926803A90813E8B50F2D
:102C100091F08347104218603504A9F080008623A4
:102C2000810842C63C1A8ED018E78084611846316C
:102C3000C303F9A826F723DF2D310854C689B861EC
:102C40003F168E11104B19070C7C2DF9A3399809EA
:102C500008430C4673308631084119082080000370
:102C60006A318C2118AA12108404D1508D63234C30
:102C700019E03148C8305B059EBE9B27C8BC783E32
:102C8000C42155B78D8008C4ADBA2FE4D12FA8F365
:102C90003AD20E3FE74AC380308F008A6681085BD4
:102CA0000545E584222089C8814009AE8D83EE95D3
:102CB000C20908430C467331042110821C70218C18
:102CC00063182A2B0434006B0306A00CA21112B067
:102CD00090378D001A27C1B1682DE4099268DD870D
:102CE000A5907E3A08423AC691ACB4268FF0D13610
:102CF0000D0413B6C5A183B4F4B70F8034BFE7F059
:102D00002C6D002188C010C461A0EC322D041B087A
:102D1000430C4673308421082D0480318C4311AA62
:102D20005054C31D4F944F3F386921F442084A5212
:102D300094B5091A00021800714EEA5655E442741F
:102D40000004D5A3EA17DFC1260342D4B4520C62B3
:102D500008430C463F3846218A20085753EF241970
:102D6000387F5C201F08430C46733084286231187A
:102D7000C822460108C6386231C2423154F50B6A96
:102D800006E82B20C8388743213E1094A58C3E02CC
:102D90007C14484E100015083F8863E11D4E418A9F
:102DA00020F8B80A9F442109F2D4F519F47D1421C2
:102DB000E83E0113E0DE46ACA350F83A8C0A33D665
:102DC0000DBD000C08430C46733008100C6118C090
:102DD0000960421882165701A82E805B2BA82F8A03
:102DE0008DA3A8BFCF4740BAA5108C5E85D44E20D6
:102DF00042D244408C8124403D045F8885F56B3F7E
:102E0000003E227300EC0944461F1637B000269C92
:102E100047E0665ADD922A8B3BFE462DA26B2102CB
:102E200046EF42EA15966B73301408430C46733034
:102E30008428842318C669A27808D63B080050303D
:102E40009A88152815FC1084A9C0040291A9FE04D3
:102E5000000118C631FC1148821A62A0254B79483E
:102E6000954682425E35BE8C218B32D12A7FAC21C1
:102E70000C3118CBE10A000043000108486230D150
:102E8000F970801408430C467330C4410863088409
:102E9000118C72812A29806B18C000007A28422A7E
:102EA000203514F431760200041A23F2F834AC22EF
:102EB000501ABF017F5E813982046040343DE08258
:102EC00010AA202B41FE36AE474510F20E4084DAA0
:102ED0003A81FC05950648EF4120C880000000A219
:102EE000118882A801CC640218006A648108618894
:102EF000CE661E08430C46733000000C8410C631A9
:102F00000C5108433454248C2A1B2021C4000A8706
:102F100043A885510421F9EA2A6338A9C210002187
:102F2000F66B9B67E008044112D0043118D45B496A
:102F300008150010C011E82C144D401021004682E5
:102F400010AB30D03F8501485773C454160E419CD6
:102F50007C01318D98FD0A00010C7C310C8B410005
:102F60001708430C46733340D0000300E219048174
:102F70000908421001ADEA0FAAA7D0BC8F80291A18
:102F80004710B2A2D739408B470988418C630C3176
:102F900099D5219E2A4D149A0713516B9A081B52FA
:102FA000692BCE747CEB6BD1F4AD1F46DF3B401434
:102FB00008430C467330C431443228C410D3F7653B
:102FC00041A3F29FC7BFFDD43EFD37A3F9FEC06DFC
:102FD0000BA23398EA5B7EA70841C5800DA9C1CE3C
:102FE000FC0BA98BF31B46CF3A00C3119CCC0C08F9
:102FF000430C467330C421431180C6386022A82593
:10300000B8F2A7B1F435E9FF18FE110C431038FFF0
:103010009AA1AF2A6A242300060D13F1D04A52C3A5
:103020001A3F520002180C80802A6CA96B10567A45
:1030300031824013FA268FACC793A00008430C4698
:103040007330C2388645A02A605CC6D1015056A0B4
:10305000F8A93ACEF0F83236DAF525235AB7429D70
:10306000B83F83B7D93E400E45A9C3505EDA152755
:1030700059DE010AE97B934888645A0C1B08430C0B
:10308000467330C638623398EA7B9F47E1FE7FFF84
:10309000E7FFFE7FFFE7FFFE7FFC216B5B0C35A0A7
:1030A0000000018AA7A9402AA02121090C46642713
:1030B000C66ABEA3584218623399800F08430C4673
:1030C0007330C63860616000086230085400200028
:1030D000270134450AA832A1D2191E85CC202CCE56
:1030E0002C0D60FF0E8531663F1E71309084212AC1
:1030F0001D1EA257C08F8738D1FE4D1021863E5D20
:10310000A2529A28157C3A1679A8E82BF84DA77C8C
:10311000593EEC0B08430C467330C63862331885B1
:103120003C540218A21902FC0869FAB7FA8AA500F1
:103130000CBA18C42143118943F2719E082A7A7A85
:10314000A7A7F47A7FE7FBC7F3FEA210421F202156
:103150005E9FCE1ADAC0A5701A08430C46733084FD
:10316000286042210840B18C6182118C70C0CB5321
:10317000302150000863430547A3D4384FCDA18ABE
:10318000A7D80210C3028ED5706C9B85F6290ABCA5
:10319000A9C953E8A421347F905FC7CFF08D7DCAC1
:1031A0007E3DC8210C3119CCC01208430C4626972D
:1031B000C6000218032440102186367CAB40090665
:1031C00031C31199329259386E63A10C2000000668
:1031D000463DCE860D5248D1F5021330D1FE1AC2BB
:1031E0003AD1BDDFE34420C6386233EE7365EEBAF0
:1031F00008000862339872DC97A31408430C4673E6
:10320000308222106318C6121080008610AE822011
:103210004240DA00086A00041104B03080000483E0
:103220005213A101EA1C0344D6422DA09F01FF21A5
:103230007F22B6B0AD092118C64080DF4C81F8135B
:10324000F9CA47ACC53500C5509004D0C7E4043A6C
:10325000008241773FC7E0015E1E05C3A110242014
:10326000C9A010601807A07751E4E81408430C4681
:103270007331084860812088288482084000322009
:10328000902399C001088428604118C70C4606A9FC
:10329000A9E18C21294B0C6657207A7A8082254F30
:1032A000907558D043C48BB8E0FB817C6BF02B2128
:1032B000044326F3C968442049F0CF3E47C340FC8D
:1032C00044C4BD1FE05C87CB1E4E802408430C46DF
:1032D00073308428623314E410800318E188CAA78D
:1032E000ABC25294BA1043AE0B995FCB599064189D
:1032F000CDF3E56219081097C4FF3A1F8024090234
:103300002C0430C46350563508000863E0A9368A9F
:103310009EE9D43F8CEEA5D8024212188C4210C30D
:10332000119CCC2A08430C467332C0200C638623C0
:103330000000021675506F2208C84210810DE3503C
:103340004B150715501044154BF2643E8687F378F1
:1033500004887E7D0AA1F86A7DE7F8D1F61FA4C330
:1033600017B7F15531DEF0318AA29C724A62A20091
:10337000263110848609C17552B8403508430C4681
:1033800073310631C30230861964240841300423A6
:1033900010AA7082DAA93CAA849BCF724FCAA321DB
:1033A000380093C918C530F05584C5A1884216B3BA
:1033B000509360D084418331E807520844583F0A53
:1033C0009F44EC347D0AA2188648C346154E31FC52
:1033D0003FC4673300080670E8F86070D8080670CC
:1033E000B8F83070D8080670F8702070D8080670E9
:1033F000A8702070D8080670F8F87020D808062049
:103400005824702058080610689038106808067014
:10341000A8F87020D80806002050B87020080620B0
:10342000702070A8240806784848584848080600C4
:10343000FC844830FC080600205088502008069084
:1034400024885004480806007078F8F8700806FCD4
:1034500084FCFC30FC080600000000000003053F6F
:10346000213F1208120A100A0E1C0E0C1E0C141A10
:1034700014161F161E131E1E1B1E1E1F1E3F213F4D
:103480003A2F3A173D173F213F181F02040A041F25
:103490000E04040E1F0A1F0A0E0E1F04110E2E2505
:1034A0002E2F2A2E262929021F02081F08150E0476
:1034B000040E150E15151B151B040604040C040040
:1034C00000000017000300031F0A1F16371A190413
:1034D000130A153A000300000E11110E000A040A27
:1034E000040E040030000404040010001804031F3C
:1034F000111F121F101D151711151F07041F171577
:103500001D1F151D01011F1F151F17151F000A0084
:10351000003200040A110A0A0A110A040115020EF7
:1035200011171E051E1F150A0E110A1F110E1F1559
:10353000111F05010E111D1F041F111F1108100F6F
:103540001F041B1F10101F061F1E040F0E110E1F3D
:1035500009060E112E1F051A121509011F011F1051
:103560001F0F180F1F0C1F1B041B031C031915131F
:10357000001F11030418111F000201022020200067
:1035800001020C121E1F120C0C12120C121F0C1A2C
:1035900014041E05242A1E1F021C141D1020201DA9
:1035A0001F0814111F101E041E1E021C0C120C3EBC
:1035B0000A040C123E1E040214160A020F120E1008
:1035C0001E0E100E1E081E120C1226281E322A264F
:1035D000041E21001F00211E040102013F213F0A99
:1035E0004E6F2053442063617264206F720A6E6FC5
:1035F000204C4F414445522E4845580A0A153A4539
:10360000786974001D20466C617368696E670A20D2
:10361000206C6F616465722E2E2E0A0A444F4E276D
:1036200054205455524E204F464621000A0A153A5E
:1036300049676E6F7265006D560A0A504C454153DA
:1036400045205455524E204F464620004C4F57209F
:103650004241545445525921200017534400161337
:103660007800161314001510200015201000540ABD
:1036700003E181867F3E186D830F0F0E0183866004
:1036800033186DC3198F1803C38E6033186DE33080
:10369000CF1803C39E603630CDE360CF3006C79E9F
:1036A0007E3E30CDB360CF300CC6F6603330D9B635
:1036B00060CF33CFCCF66061B0DB1E60CF30D86C0A
:1036C000E6C061B0DB1E618F19986CC6C063B19B08
:1036D0000E330F0FB078C6FF7E1F1B061E0F0500AE
:1036E000893008023802497868140000F6E8DBCF18
:1036F000C3B8AEA49B928A827B746E68625C575298
:103700004E4945413E3A3734312E2C292725232175
:103710001F1D1C1A1917161514131211100F0E0D58
:103720000C0B0A090807064500680100000500683F
:1037300001380100000500380168010000453741EB
:10374000370101FF030101F7030000000800020137
:103750000000030407000000000000000001020454
:103760000810204080010204081020010204081003
:1037700020040404040404040402020202020203FA
:1037800003030303030000000023002600290000B8
:10379000000000250028002B000000000024002766
:1037A000002A0000B42411241FBECFEFD8E0DEBFF2
:1037B000CDBF12E0A0E0B1E0E8EAF5E702C0059075
:1037C0000D92A837B107D9F726E0A8E7B2E001C00B
:1037D0001D92AF33B207E1F717E3C6EAD7E304C09F
:1037E0002297FE010E949E3AC43AD107C9F70E946F
:1037F0004E370C94D23A0C9400000C94BC3A0C94C2
:10380000C43A1092850284E680930B0110928102E3
:1038100010928002109283021092820210927D0216
:1038200010927F0208951F93CF93DF93162F20915C
:103830007B0230917C02E82FF0E0EE0FFF1FE45F87
:10384000FE4FC90137FD079643E0959587954A9548
:10385000E1F70190F081E02DE80FF91FC491319656
:10386000E491D0E0DC2FCC27CE0FD11DE12FF0E08A
:10387000C90168E070E00E94473A40E150E0481B0F
:10388000590B4E1B5F0B02C0D595C7954A95E2F7C1
:103890002E0F3F1F30937C0220937B0281E090E04B
:1038A00002C0880F991F1A95E2F701978C23DF91C8
:1038B000CF911F910895482F8091790290917A02BB
:1038C00064E170E00E94473A77279C013327493032
:1038D000E9F188F44730D1F1483009F043C08EE077
:1038E000829FF001839FF00D1124E60FF71FE05730
:1038F000FD4F88E429C04C3081F04D30D1F04A3082
:1039000089F58EE0829FF001839FF00D1124E60F70
:10391000F71FE057FD4F8AE417C08EE0829FF00149
:10392000839FF00D1124E60FF71FE057FD4F8AE843
:103930000BC08EE0829FF001839FF00D1124E60FF3
:10394000F71FE057FD4F88EC808308958EE0829F3B
:10395000F001839FF00D1124E60FF71FE057FD4F94
:10396000408308958EE0829FF001839FF00D112423
:10397000E60FF71FE057FD4F40834B3041F4309383
:103980008F0220938E0270938D0260938C020895B3
:10399000CF92DF92EF92FF920F931F93CF93DF931B
:1039A000F82E1092860210927C0210927B021092E6
:1039B0007A021092790268E00E94131C80938702B9
:1039C000C4E1D0E0EEE0EE2E2091790230917A024F
:1039D000283131400CF04DC061E08F2D0E94131C46
:1039E0008823B1F166E08F2D0E94131C082F63E03D
:1039F0008F2D0E94131C73E0C72EC80ED12C10E02F
:103A0000DC1410F72091790230917A02283181E09C
:103A10003807E4F4C901801B910BBE010E94473AAC
:103A2000E89EF001E99EF00D1124E60FF71FE05724
:103A3000FD4F80810E945B1C2091790230917A02B7
:103A40002F5F3F4F30937A0220937902D394D8CFDF
:103A500064E08F2D0E94131C0E945B1C2091790250
:103A600030917A022F5F3F4F30937A022093790290
:103A7000ABCFDF91CF911F910F91FF90EF90DF902F
:103A8000CF90089590918502953920F580917E021E
:103A9000811106C0809180028F5F8093800205C0F3
:103AA000809182028F5F80938202209181028091B7
:103AB0008002821708F4822F809381022091830272
:103AC00080918202821708F4822F809383029F5F85
:103AD00090938502809185020C94C81C0F931F93CC
:103AE000CF93DF9380E090E00E94FD1B813D09F0C1
:103AF0004AC081E090E00E94FD1B863609F043C079
:103B000082E090E00E94FD1B8933E9F583E090E0BC
:103B10000E94FD1BC1E0811101C0C0E0C0937E0284
:103B200084E090E00E94FD1BD82F8093800285E006
:103B300090E00E94FD1B082F8093810286E090E0B8
:103B40000E94FD1B80930B0188E090E00E94FD1B0A
:103B5000182F8093820289E090E00E94FD1B902F35
:103B60000D1708F49D2F90938102811708F4812F7F
:103B700080938302C111D12FD0938502C11101C05E
:103B8000892F80938402DF91CF911F910F91089527
:103B900063E970E088EA93E00E9465310E946E1D3F
:103BA000809185020C94C81C88EA93E00E94E2315F
:103BB0000E94C81D1092C003089561ED80E090E05E
:103BC0000E94FF1B66E681E090E00E94FF1B69E314
:103BD00082E090E00E94FF1B60917E0283E090E013
:103BE0000E94FF1B6091800284E090E00E94FF1B16
:103BF0006091810285E090E00E94FF1B60910B01C3
:103C000086E090E00E94FF1B6091820288E090E0D5
:103C10000E94FF1B6091830289E090E00C94FF1BDF
:103C20009FEF980F923168F49FEF960F9C3048F405
:103C30009EE0899FF0011124E60FF11DE057FD4F32
:103C40004083089540918E0250918F0220918C0202
:103C500030918D029EE0949FF001959FF00D11240C
:103C6000E20FF31FE057FD4F1082480F511D87FDF3
:103C70005A9550938F0240938E02260F311D67FD97
:103C80003A9530938D0220938C02949FF001959F7A
:103C9000F00D1124E20FF31FE057FD4F8BE08083FE
:103CA0000895662321F08DEC93E00C94113548E0E3
:103CB00062E082EB93E00E94F0258823B1F08091CE
:103CC0008E0290918F02029620918C0230918D028B
:103CD0004EE0489FF001499FF00D1124E20FF31FC1
:103CE000E057FD4F80818823F9F048E060E082EBE7
:103CF00093E00E94F025882361F180918E029091DB
:103D00008F02029720918C0230918D024EE0489FE5
:103D1000F001499FF00D1124E20FF31FE057FD4F12
:103D20008081882361F0089582E0808360E081E0F3
:103D30000E94221E8DEC93E00E94FB34D6CF82E0DD
:103D4000808360E08FEF0E94221E8DEC93E00C9444
:103D5000FB34089580918C02E0918E029EE0E99FF1
:103D6000F0011124E80FF11DE057FD4F8CE0808336
:103D700081E080937F0280910B01815080930B0141
:103D80000895BF92CF92DF92EF92FF920F931F930D
:103D9000CF93DF93E82EF62E082F10E0C80101978D
:103DA000C62FD0E0DE0111974EE0489FB001499F39
:103DB000700D1124CB018A0F9B1F80579D4FFC0172
:103DC00080818B3009F447C0CB018C0F9D1F805739
:103DD0009D4FFC0180818B30F1F19E012F5F3F4FA1
:103DE000FB01E20FF31FE057FD4F80818B3099F10B
:103DF000409FB001419F700D1124CB018A0F9B1F82
:103E000080579D4FFC0180818B3029F1FB01E20F2F
:103E1000F31FE057FD4F80818B30E9F0C801019618
:103E2000489FF001499FF00D1124AE0FBF1FA0570E
:103E3000BD4F8C918B3079F0DF01AC0FBD1FA057C7
:103E4000BD4F8C918B3039F0E20FF31FE057FD4FDF
:103E500080818B3011F40E94AA1EBB24BA94BE0C40
:103E600040E0DD24D394DF0C6D2D8B2D0E94101EBD
:103E700040E06D2D8E2D0E94101ECC24C394CE0CDC
